:10F800000C943E7C0C94627C0C94627C0C94627C24
:10F810000C94627C0C94627C0C94627C0C94627CF0
:10F820000C94627C0C94627C0C94627C0C94627CE0
:10F830000C94627C0C94627C0C94627C0C94627CD0
:10F840000C94627C0C94627C0C94627C0C94627CC0
:10F850000C94627C0C94627C0C94627C0C94627CB0
:10F860000C94627C0C94627C0C94627C0C94627CA0
:10F870000C94627C0C94627C0C94627C11241FBEFC
:10F88000CFEFD0E1DEBFCDBF11E0A0E0B1E0E6E612
:10F89000FDEF02C005900D92A030B107D9F711E03D
:10F8A000A0E0B1E001C01D92A030B107E1F70E94D5
:10F8B000707C0C94B27E8FEF90E19EBF8DBF1124BF
:10F8C0001FBE0EC00C94007C8093CE008091C800B7
:10F8D00086FFFCCF8091C80080648093C8000895A3
:10F8E000CDB7DEB7CD51D140DEBFCDBF4D9B06C1F8
:10F8F0001092CD0083E08093CC0088E18093C90012
:10F900006624772400E09924AA24BB2444245524A7
:10F910001E010894211C311C10E0EE24FF2480916C
:10F92000C80087FD0CC089B190E0FC01E072F07066
:10F9300085FDF5CF09958091C80087FFF4CF209110
:10F94000CE00133009F481C0143068F4113009F48A
:10F9500089C0123008F480C0822F90E0F82EEE2487
:10F96000022713E0DCCF153009F461C0153008F42C
:10F9700057C0163009F44FC0173089F6298123315A
:10F9800009F418C1243108F075C0263009F49DC16E
:10F99000273008F0A6C0223009F4CDC0233009F486
:10F9A000F2C0213009F4D2C080EC8A8392E0C92EE3
:10F9B000D12C8824EE2400E082E0F82E12E08BE1C6
:10F9C0000E94647C892D0E94647C802F0E94647C4C
:10F9D000812F0E94647C8EE00E94647C05E10925F1
:10F9E0000E250F25C114D10471F07101F701119199
:10F9F0007F01812F0E94647C01270894C108D108EF
:10FA0000C114D10499F7802F0E94647C882009F0EA
:10FA100075C0939481CF021709F4B0CF10E07FCF67
:10FA20002E30E1F7022715E06624772478CFF10124
:10FA3000E60DF71D20830894611C711C02276E14CB
:10FA40007F0409F06CCF16E06ACF822F90E0E82A9D
:10FA5000F92A022714E063CF2B3109F060CF11E0BF
:10FA60000BE15DCF213011F09216C1F60227922EE4
:10FA700012E055CF283109F4FBC0293108F047C006
:10FA8000253109F497C02531A8F58A8190E0582FD7
:10FA900044278B8190E0482B592BA3E0CA2ED12C10
:10FAA000C40ED51E1A82243109F41BC1BA01950176
:10FAB000DE01139621BD832F992782BD2F5F3F4F13
:10FAC000F89A80B58D9361507040A1F7A40EB51ED1
:10FAD0001C928D2D9927E82E082FFC2C1C2D882494
:10FAE0006ECF213109F410C1223110F11A82442461
:10FAF00055245CCF263109F057CFC7CF81E18093E1
:10FB00005700E89511241F921F920895FFCF2B31C3
:10FB100009F412C12D3109F4FAC02A3109F044CF99
:10FB20001A8289E0E1E0F0E0809357008491AAC056
:10FB3000203109F039CF88241A82F2E0CF2ED12C5F
:10FB4000EE2400E0E2E0FE2E12E039CF1A8288E0D7
:10FB50008B8381E48C8386E58D8382E58E8389E4C3
:10FB60008F8383E5888780E589878FE58A8782E3AD
:10FB70008B870BE0C02ED12C8824EE2400E01BE004
:10FB8000F12E1BE01CCF8A81813909F48BC08239A8
:10FB900009F484C0803909F483C080E01A828B8321
:10FBA000B3E0CB2ED12C8824EE2400E0A3E0FA2E83
:10FBB00013E005CF8A8190E0782F66278B8190E053
:10FBC000682B792B2331B9F0AB019501FE013B96EF
:10FBD00021BD832F992782BD2F5F3F4F819180BD2B
:10FBE000FA9AF99AF999FECF4150504089F7A60E3A
:10FBF000B71E1A82DBCE40E0441648EF540660F48C
:10FC000083E0F20180935700E89507B600FCFDCF32
:10FC100080E091E0480E591ED5018BE0E82EF12CD2
:10FC2000EC0EFD1EF7018081218142E050E0E40EE0
:10FC3000F51E41E030E0322F222790E0282B392BAF
:10FC40000901FD0140935700E89511241296625076
:10FC5000704041F785E0F50180935700E89507B6BD
:10FC600000FCFDCF81E180935700E8955D01C1CF95
:10FC70008B818035C9F089E0E3E0F0E080935700A4
:10FC800084911A828B831C8274E0C72ED12C882425
:10FC9000EE2400E064E0F62E14E091CE8AE07ECF00
:10FCA0008FE07CCF82E07ACF8C81883039F089E098
:10FCB000E0E0F0E0809357008491E3CF89E0E2E058
:10FCC000F0E0809357008491DCCF8C8190E0B82ED7
:10FCD000AA248D8190E0A82AB92AAA0CBB1C1A82FA
:10FCE00065CEDE011396F501859194918C93892F51
:10FCF0009927FD018183129682E090E0A80EB91E3B
:10FD00004250504081F7E4CE8824839415CF9D81E2
:10FD10009033B9F080E01A821B829C839E819D8380
:10FD20008E831F8297E0C92ED12C8824EE2400E018
:10FD300087E0F82E17E043CE8D81882339F48EE1D9
:10FD4000A0CF8F81882331F48EE1E5CF813031F06F
:10FD50008AE097CF813021F08AE0DDCF86E991CF2C
:06FD600086E9D9CFFFCFB8
:040000030000F80001
:00000001FF
